:0200000480007A
:100000006F00C004732F2034930F8000630AFF0336
:10001000930F90006306FF03930FB0006302FF038A
:10002000170F0080130F0FFE63040F0067000F000F
:10003000732F203463540F006F004000136E9E53E3
:10004000171F00002320CFFD6FF09FFF732540F1A5
:100050006310050073251030635805000F00F00F82
:10006000130E100073000000130E00009702000032
:10007000938282F973905230735020307350303035
:1000800073504030970200809382C2F7638C020065
:10009000739052109302B01A739022307323203061
:1000A000E39E62F873500030970200009382420191
:1000B00073901234732540F17300203097200000B4
:1000C000938040F41301A00A239020008391000044
:1000D000930EA00A130E2000639ED14597200000C6
:1000E000938040F237B1FFFF130101A0239120005C
:1000F00083912000B7BEFFFF938E0EA0130E300039
:10010000639AD143972000009380C0EF3711EFBE70
:10011000130101AA2392200083A14000B71EEFBE65
:10012000938E0EAA130E40006396D14197200000D3
:10013000938040ED37A1FFFF1301A100239320001E
:1001400083916000B7AEFFFF938EAE00130E500098
:100150006392D13F972000009380A0EB1301A00A87
:10016000239D20FE8391A0FF930EA00A130E600032
:100170006392D13D972000009380A0E937B1FFFF43
:10018000130101A0239E20FE8391C0FFB7BEFFFF95
:10019000938E0EA0130E7000639ED139972000003D
:1001A000938020E737110000130101AA239F20FE4E
:1001B0008391E0FFB71E0000938E0EAA130E8000FD
:1001C000639AD137972000009380A0E437A1FFFF06
:1001D0001301A1002390200083910000B7AEFFFF20
:1001E000938EAE00130E90006396D13597200000D9
:1001F000938040E23751341213018167138200FE6D
:100200002310220283910000B75E0000938E8E6758
:10021000130EA0006390D13397200000938080DFFD
:1002200037310000130181099380B0FFA3932000B0
:1002300017220000130222DE83110200B73E0000E5
:10024000938E8E09130EB0006396D12F130EC0004B
:1002500013020000B7D0FFFF9380D0CD172100001C
:10026000130141DA2310110083110100B7DEFFFFF3
:10027000938EDECD6390D12D1302120093022000E5
:10028000E31A52FC130ED00013020000B7C0FFFFA8
:100290009380D0CC172100001301C1D613000000B9
:1002A0002311110083112100B7CEFFFF938EDECC06
:1002B0006392D1291302120093022000E31852FC2A
:1002C000130EE00013020000B7C0FFFF9380C0BC14
:1002D00017210000130101D31300000013000000D8
:1002E0002312110083114100B7CEFFFF938ECEBCC5
:1002F0006392D1251302120093022000E31652FCF0
:10030000130EF00013020000B7B0FFFF9380C0BBD4
:1003100013000000172100001301C1CE23131100A8
:1003200083116100B7BEFFFF938ECEBB6394D121D2
:100330001302120093022000E31852FC130E000176
:1003400013020000B7B0FFFF9380B0AB13000000B2
:1003500017210000130101CB13000000231411002A
:1003600083118100B7BEFFFF938EBEAB6394D11D96
:100370001302120093022000E31652FC130E100128
:1003800013020000B7E0FFFF9380B0AA1300000043
:1003900013000000172100001301C1C6231511002E
:1003A0008311A100B7EEFFFF938EBEAA6394D1190B
:1003B0001302120093022000E31652FC130E2001D8
:1003C00013020000172100001301C1C3B720000071
:1003D000938030232310110083110100B72E0000F9
:1003E000938E3E236398D1151302120093022000CE
:1003F000E31A52FC130E3001130200001721000013
:10040000130141C0B7100000938030221300000098
:100410002311110083112100B71E0000938E3E228C
:10042000639AD1111302120093022000E31852FCC8
:10043000130E40011302000017210000130181BCBC
:10044000B71000009380201213000000130000007A
:100450002312110083114100B71E0000938E2E124B
:10046000639AD10D1302120093022000E31652FC8E
:10047000130E50011302000017210000130181B870
:100480001300000093002011231311008311610059
:10049000930E20116390D10B1302120093022000DF
:1004A000E31C52FC130E6001130200001721000030
:1004B000130141B513000000930010011300000068
:1004C0002314110083118100930E10016394D1074E
:1004D0001302120093022000E31A52FC130E700163
:1004E00013020000172100001301C1B11300000026
:1004F00013000000B7300000938010002315110096
:100500008311A100B73E0000938E1E006394D103B7
:100510001302120093022000E31652FC37C50000BC
:100520001305F5EE972500009385C5AD2393A5002F
:10053000631CC0010F00F00F63000E00131E1E00AD
:10054000136E1E00730000000F00F00F130E10005A
:1005500073000000731000C00000000000000000E5
:10056000000000000000000000000000000000008B
:10057000000000000000000000000000000000007B
:040580000000000077
:1010000000000000000000000000000000000000E0
:1010100000000000000000000000000000000000D0
:1010200000000000000000000000000000000000C0
:1010300000000000000000000000000000000000B0
:081040000000000000000000A8
:10200000EFBEEFBEEFBEEFBEEFBEEFBEEFBEEFBE68
:10201000EFBEEFBE00000000000000000000000066
:040000058000200057
:00000001FF
